:1000000042C082C15BC05AC059C058C057C056C018
:1000100055C054C053C052C051C050C04FC04EC054
:100020004DC04CC04BC04AC049C048C047C046C084
:1000300045C044C0090212000101008019090400F2
:1000400000000000000012011001FF000008C016AF
:10005000DC050201010200010E03550053004200BD
:100060006100730070001C037700770077002E009A
:10007000660069007300630068006C002E00640075
:1000800065000403090411241FBECFEFD2E0DEBFD8
:10009000CDBF11E0A0E0B1E0E0E2FEE002C00590DB
:1000A0000D92A230B107D9F711E0A2E0B1E001C092
:1000B0001D92A334B107E1F796D6B1C6A1CF1F9325
:1000C000CF93DF936091270116160CF580912401E0
:1000D000C7E3D1E0C81BD109635020E010E880914C
:1000E00023018D3209F44CC08091020187FD09C0C3
:1000F000CE01B8D52FEF821709F470C0811120E02E
:1001000010E01093020120930101109227018091C9
:10011000000184FF27C0809101018F3F19F1682FF2
:10012000893008F050C0861B809301011BE4809148
:10013000020180FD13EC8F5F80930201A8E1B1E022
:1001400087FD56C0662309F04EC060E070E0C62F00
:100150006930D8F19EE18FEF809301011093170170
:10016000909300019AE083B1837011F49150D9F714
:10017000992309F0A1C090932801909322019CC07B
:100180008AE580930001683009F0BBCF88818076D2
:1001900009F048C040E251E0209320018981882382
:1001A00009F04CC02093210122E050932601409396
:1001B00025018F81882309F0A4CF8E81821708F052
:1001C000A0CF282F9ECF68E0AECF88E191E098D0F5
:1001D0009C2F9C5FC83008F0C1CFBDCF8EE18093CB
:1001E000000110E08ECFCD01F0D4682F7727AFCF7C
:1001F000E0912501F091260186FF0DC0962F03C0E6
:1002000084918D9331969150D8F7F0932601E09325
:10021000250177279CCF962F02C081918D93915015
:10022000E0F7F3CFCE01A1D3282F8F3F09F0C1CF44
:10023000888187FF65CF2E8110E063CF853059F02C
:10024000863069F08830D9F08930E9F08A3009F0D9
:10025000B0CF21E0AACF8A8180932801AACF10ECE9
:100260008B818130A1F08230F9F0833009F0A1CF89
:100270008A81882381F442E850E024E096CF4AE264
:1002800051E021E092CF8A8180932A0192CF46E407
:1002900050E022E18ACF813059F0823009F089CFD5
:1002A00048E550E02EE081CF44E350E022E17DCFED
:1002B00046E650E02CE179CFDF91CF911F91089570
:1002C00080916900836080936900E89A0895A82F5F
:1002D000B92F8FEF9FEF41E050EA615070F02D9100
:1002E00038E0722F782796958795269570FF02C083
:1002F000842795273A95A9F7F0CF80959095089592
:10030000E6DF8D939D930895CF93CFB7CF93189B3E
:10031000FECF189B09C0189B07C0189B05C0189BEF
:1003200003C0189B01C09EC0DF93C0912401DD274C
:10033000C55DDE4F189B02C0DF91EBCF2F930F936B
:100340001F9303B12FEF00FB20F94F933F9313B19D
:100350004FEF012700FB21F93BE031C04E7F012F19
:1003600013B1216028C0102F4D7F2260000003B11F
:1003700029C04B7F2460012F000013B12BC013B1A3
:10038000477F28602AC04F7E03B120612CC04F7D7B
:1003900013B120622FC04F7B03B1206432C04227CB
:1003A00003B149934FEF0000102710FB20F913B160
:1003B0001370A9F1297F91F2012700FB21F903B104
:1003C000237F89F23150F0F1102710FB22F913B18D
:1003D000277E79F2012700FB23F92F7C81F203B1FC
:1003E000102710FB24F92F7971F200C013B10127F7
:1003F00000FB25F92F7359F200C003B1102710FB41
:1004000026F9223040F200C013B1012700FB27F982
:10041000243028F64F77206813B10000F9CF3B5005
:100420003195333011E01CBBB8F0C31BD0400881BC
:10043000033C41F10B3431F11981412F1F77209199
:100440002201121731F4093691F10D3279F0013E93
:1004500069F02227209329013F914F911F910F911D
:100460002F91DF91CF91CFBFCF91189500932901A4
:100470003F914F911F910F912F91DF91CCB3C0FD10
:1004800046CFF0CF00912901002331F310912701CD
:10049000112349F534304AF13093270100932301A9
:1004A000109124013BE0311B309324011EC00091C8
:1004B00027010130C4F40AE53091000134FD17C072
:1004C00000930001C7E1D1E016C0052710E005B98F
:1004D0001FC0052722C0052727C005272CC00527D8
:1004E00010E005B933C04AE503C042ED01C0432F17
:1004F000C4E1D0E032E014B11360289A05B114B918
:100500005F9353E020E820FF052705B9279517954D
:100510001C3FD8F620FF0527279505B917951C3FE6
:10052000C0F620FF05272795179505B91C3F98F6BB
:1005300020FF0527279517951C3F05B970F600C0C9
:10054000499120FF052705B9279517951C3F38F6D7
:1005500020FF0527279505B917951C3F38F520FF83
:1005600005272795179505B91C3F10F520FF05278E
:10057000279517951C3F05B9E8F4242F3A9519F6ED
:100580000C7F5F9105B900C010912801C651D04081
:1005900011F01093220111E01CBB016014B11C7F0B
:1005A000402F4C7F05B914B945B956CF0527D3CF95
:1005B0000527D8CF0527DDCF3B98439A00000000E0
:1005C000339904C082E58CBD1DBC08953A9A4298C7
:1005D00000000000339B07C082E58CBD81E08DBD2B
:1005E0003A98429A089583E58CBD1DBC3A98429A88
:1005F0000895882339F48EE293E09093420180932A
:10060000410108958BE493E090934201809341016E
:10061000089596B586B5891B8C30E0F308952C9A21
:100620003D9A459884B18C6284B92A982D98F1DF5F
:100630002A9AEFDF2A9880914101909142018B54D0
:10064000934009F00895B8DF089584B1837D84B99B
:1006500085B1837D85B93D981CBC08950F931F9388
:10066000CF93C82F00E017E00CC02B98CC0F000FE1
:100670001C990F5FCEDF2D9ACCDF2D98115017FDFE
:1006800004C0C7FFF2CF2B9AF1CF802F9927CF91CB
:100690001F910F9108958EBD0DB407FEFDCF8EB54D
:1006A000992708951F93CF93CFE103C0C150CF3F47
:1006B00051F1E0914101F09142018CEA0995E091FC
:1006C0004101F091420183E50995E0914101F091EA
:1006D000420180E00995182FE0914101F09142011B
:1006E00080E00995133591F01CBC2D9A92DF2D986E
:1006F00090DF80914101909142018B549340B1F67B
:100700005BDFC150B0F681E090E002C080E090E095
:10071000CF911F910895EF92FF920F931F937B014A
:100720008C01862F8170880F880F880FE09141011E
:10073000F091420180620995D801C70129E0B69580
:10074000A795979587952A95D1F7E0914101F0916A
:100750004201099516950795F794E794E0914101B8
:10076000F09142018E2D0995E0914101F0914201F5
:1007700080E0099599271F910F91FF90EF900895C0
:10078000CF92DF92EF92FF921F93CF936B017C0188
:10079000C42F122F862F8170880F880F880FE09149
:1007A0004101F091420180640995D701C60149E0F9
:1007B000B695A795979587954A95D1F7E091410110
:1007C000F09142010995D701C601B695A795979575
:1007D0008795E0914101F09142010995E091410135
:1007E000F09142018C2F09951123B1F0CF3791F090
:1007F0001EE1C6B5C701B6018EDF8F3769F486B535
:100800008C1B8D3310F0C6B51150112399F781E080
:1008100090E004C08FE09CD080E090E0CF911F91E9
:10082000FF90EF90DF90CF900895CF92DF92EF92FC
:10083000FF921F93CF936B017C01142FE091410134
:10084000F09142018CE40995D701C60169E0B695A3
:10085000A795979587956A95D1F7E0914101F09119
:1008600042010995D701C601B695A7959795879539
:10087000E0914101F09142010995E0914101F0912F
:10088000420180E009951F3F91F01EE1C6B5C70106
:10089000B60141DF8F3F69F486B58C1B8D3310F0B4
:1008A000C6B51150112399F781E090E004C08FE0A4
:1008B0004FD080E090E0CF911F91FF90EF90DF90BC
:1008C000CF9008950F931F938C01E0914101F09117
:1008D000420180EA0995812F9927E0914101F09129
:1008E00042010995E0914101F0914201802F099563
:1008F000E0914101F091420180E0099599271F9113
:100900000F910895FF920F931F938C01F62EE091A3
:100910004101F091420180EC0995812F9927E091E6
:100920004101F09142010995E0914101F0914201AC
:10093000802F0995E0914101F09142018F2D099599
:100940008EE106D080E090E01F910F91FF90089516
:10095000382F20E0231740F496B586B5891B8C33D9
:10096000E0F32F5F2317C0F308951F93CF93DF9316
:10097000EC0110E089818130B9F0823009F49FC028
:10098000833009F49FC08430B9F0873009F471C016
:10099000853009F4FAC08630C1F1883009F4C9C045
:1009A000893009F006C1F6C0329B812F22DE1092F9
:1009B000060135DE4198FDC0809106018823A1F42F
:1009C0008B819927982F88272A813327822B932B75
:1009D000AA2797FDA095BA2F80930F01909310013D
:1009E000A0931101B09312018F819927982F882726
:1009F0002E813327822B932B909304018093030144
:100A000082E0809305011FEFD4C080910601882306
:100A100009F47AC08C81482F5527509314014093D4
:100A200013012D812F70209315018D819927807FCF
:100A3000907082959295907F9827807F9827840F59
:100A4000951F909314018093130120FF04C080919F
:100A50001301809316018F819927982F88272E8163
:100A60003327822B932B909304018093030181E021
:100A7000C8CF809106018823A1F48B819927982FF4
:100A800088272A813327822B932BAA2797FDA095AD
:100A9000BA2F80930F0190931001A0931101B0938E
:100AA00012018F819927982F88272E813327822B37
:100AB000932B909304018093030183E0A2CFC5DDC3
:100AC000419A77C0E0914101F09142018A810995F4
:100AD00080930701E0914101F09142018B810995DA
:100AE00080930801E0914101F09142018C810995C8
:100AF00080930901E0914101F09142018D810995B6
:100B000080930A0114E055C08B819927982F88277C
:100B10002A813327822B932BAA2797FDA095BA2FE2
:100B200080930F0190931001A0931101B0931201D3
:100B300071CF809106018823A1F48B819927982F8A
:100B400088272A813327822B932BAA2797FDA095EC
:100B5000BA2F80930F0190931001A0931101B093CD
:100B600012011092140110921301109315018F813C
:100B70009927982F88272E813327822B932B9093A8
:100B800004018093030184E03CCF8CDD8093070156
:100B900011E00FC081E0809306018A819B81AC81C6
:100BA000BD8180930F0190931001A0931101B09328
:100BB000120187E091E09093260180932501812F17
:100BC0009927DF91CF911F910895EF92FF921F9384
:100BD000CF937C01162F90910501892F825082308E
:100BE000D0F5C0E0C61710F12FC080910F01909191
:100BF000100168DEF701EC0FF11D808380910F0179
:100C000090911001A0911101B09112010196A11DC6
:100C1000B11D80930F0190931001A0931101B09327
:100C20001201CF5FC11780F4909105019230E9F66F
:100C300080910F0190911001A0911101B0911201CA
:100C4000BC01CD0168DDD6CF183010F4109205013B
:100C5000812F992702C08FEF90E0CF911F91FF90D5
:100C6000EF900895BF92CF92DF92EF92FF920F9391
:100C70001F93CF93DF936C01062FBB2420910501B6
:100C8000213019F0243009F0A2C010E0101708F04C
:100C90009BC0213009F05FC0809113019091140135
:100CA000892B09F064C0C12FDD27FE01EC0DFD1D6D
:100CB00080910F0190911001A0911101B09112014A
:100CC0004081BC01CD015CDD809103019091040164
:100CD00001979093040180930301892B09F51092E9
:100CE00005018091150181FF19C080911601282FFF
:100CF000332780911301909114012817390771F05F
:100D0000CC0DDD1D80910F0190911001A09111017A
:100D1000B09112014881BC01CD0187DDC1E0BC2E3C
:100D200080910F0190911001A0911101B0911201D9
:100D30000196A11DB11D80930F0190931001A09306
:100D40001101B09312011F5F1017F0F520910501FA
:100D5000213009F4A1CFC12FDD27FE01EC0DFD1DCF
:100D6000608180910F0190911001CCDDADCFC12F3A
:100D7000DD277E01EC0CFD1C80910F01909110018C
:100D8000A0911101B091120120E0F7014081BC0156
:100D9000CD01F6DC809116018150809316018823E5
:100DA00009F092CF80910F0190911001A091110153
:100DB000B0911201F7014081BC01CD0136DD809177
:100DC00013018093160180CF8B2D992702C08FEFDE
:100DD00090E0DF91CF911F910F91FF90EF90DF9006
:100DE000CF90BF900895CFEFD2E0DEBFCDBF1BB84C
:100DF00015B88BEF8AB98FEF84B990E09150F1F775
:100E00008150D9F784B993E097B98EEF88B995BD31
:100E100081E0EFDB55DA789452D951D9FDCFFFCF7D
:020E20005AFF77
:00000001FF
